:020000009D2839
:08000800002882073334333471
:100010003234203406340C34013402342008820790
:100020000034013402340334043405340634073414
:10003000083409340A340B340C340D340E340F34C4
:100040008207542BF52BEA2C592C7E2B132C1D2DBB
:10005000862CA52B2B2C3A2DAA2CCC2B422C552DA3
:10006000CA2C8207E12A162B462A3A2B82075334E0
:100070007434613474346E34233431342034233492
:1000800032342034233433342034233434340034B1
:100090008207533465347234763420344D346F34EF
:1000A0006434653420345034613467342F3452342E
:1000B000673400348207203445346D34653472343B
:1000C000673465346E346334793420345334743493
:1000D0006F3470342134003482074D3469346E3407
:1000E00069344434433443342034533474346134F5
:1000F000743469346F346E342034003482075634DB
:1001000065347234733469346F346E34203435346A
:100110002E34363400348207543472346E346F34E3
:100120007534743420344334743472346C34203471
:100130004D346F34643465340034C1209025392740
:10014000D408031DB32849273527A826AB26AE2699
:10015000B1264927DE26E226E626EA266418492249
:1001600056184922A028392735274927BD20D40809
:100170000319A328D6184922B4284826C1193E26B7
:10018000080007309F0083162C30850086018312FB
:100190008601213084006030A0008001840AA00B19
:1001A000CD2846308400B701370889258000840AAD
:1001B000B70A06303706031DD428B4229030CC008D
:1001C000CD00CE00CF008030D700D900F830D80065
:1001D000DA00DD0A4130E1000800C1180800D40847
:1001E000031D0800C1140430AE0056180800D40ADC
:1001F000C0303226B70137085A20B70A003E03192B
:1002000003291A26FB284A08A800CA01C522420869
:10021000EA004308EB004408EC004508ED004130DB
:10022000C200C300C400C5006E1CC216EE1CC3167B
:100230006E1DC416EE1DC5160A30A5001930B70094
:10024000BF27851D3D294927A826AB26AE26B12606
:100250004927A50B1E292808CA0056106A08C200A3
:100260006B08C3006C08C4006D08C500C522B42526
:10027000F825D401C0304D23F82DC0304D23C110D6
:10028000D4012808CA004429C1180800C114043048
:10029000AE00B4225408D40A3128D6196C2937226A
:1002A000D615D625C03032264C3084000430BA0032
:1002B0002D3000182A301A262D3080182A301A26A0
:1002C0002D3000192A301A262D3080192A301A268E
:1002D000840ABA0B58290800D601D401B425F82D98
:1002E000DF0ADF0ADF0ADF0ADF0ADF0ADF0ADF0AC6
:1002F000DF0A6008DB00DC00DB0DDB0DDB0D5C0DD5
:100300005B075F07CB0058105A105F08E000DF0161
:1003100008008030322652301A2665301A266330A3
:100320001A269E29561C0800D6190800803032264D
:1003300050301A266C301A2679301A26332752305C
:100340001A2674301A2665301A26332761081A26B1
:1003500033275D08282633274B087F3928267C3031
:10036000CB1B2F301A26E82956190800DD0A043065
:100370005D0767078925A90803195615CB000800F2
:100380005611DD0BB729DD0A080061085A3A031936
:100390000800E10AD1296108413A03190800E10384
:1003A000D1295611E701413061020319E129E80022
:1003B000053067078925E70AA908031DD829E80B36
:1003C000D8290130DD00053067078925CB000800FA
:1003D0007B30E900B4000530B20032088925A90855
:1003E000031DE903B20AB40BED29C03032265B309D
:1003F0001A2669082C265D301A2ECB080319102AFC
:100400005818CB1704305D076707EA008925A9084B
:10041000031919224B08A2006A0870255611B42945
:1004200004305D076707EA008925A908031D282213
:1004300008006A08803CEB008030E5006508E503B1
:1004400065088925A200650A7025EB0B1F2A0800A4
:100450006A08803CEB006A08E5006508E50A650863
:100460008925A20065037025EB0B2E2AB729B5015B
:1004700001301A26362EC1180800C1140430AE000F
:10048000561C432A4D293722561492293722D61456
:1004900089296418672A59085702031D522A5A08E5
:1004A0005802031D5622D61C922989295708D900C3
:1004B0005808DA005B275708BD00B90068278F2766
:1004C0005808BE00B9006827BF01C001752FE608B3
:1004D000031D6E2A05306707E500DD01E60A6608A0
:1004E000323A031D0800E601E60A65088925E50A97
:1004F000A9080319852ADD0A7D2ACB00A91F832AB2
:10050000B1224927522A8B22812A6410E601DD0894
:100510000319DD0A08005810CB134B08033EDB001B
:10052000D701D717D81058110310DB0C0318D814B3
:100530000310DB0C031858150310DB0C03185714B9
:100540000310DB0C0318D7140310DB0C031857152A
:100550000310DB0C0318D7150310DB0C0318571618
:1005600008005814CB178D2A60304A1A8030C20018
:100570006030CA1A8030C30060304A1B8030C4002B
:100580006030CA1B8030C500EE01E030C205C305F3
:10059000C405C5054A1C4216CA1C43164A1D44160A
:1005A000CA1D451680304A1AC205CA1AC3054A1B1D
:1005B000C405CA1BC505D001D101D201D301AD01CB
:1005C000080080303226B70137083620B70A003ECF
:1005D0000319EC2A1A26E42AC030322641301A26A2
:1005E00064301A2664301A2672301A2620304A1CCB
:1005F0003C304A1A3E301A26460828262030CA1CAB
:100600003C30CA1A3E301A264708282620304A1D98
:100610003C304A1B3E301A26480828262030CA1D86
:100620003C30CA1B3E301A264908282E803032261C
:10063000B70137084820B70A003E0319212B1A26B4
:10064000192BD20AC030322643301A2656301A26C9
:100650003A301A262D08AC005008013E2C262D30C9
:100660001A2651082C263327520828262D301A2600
:100670005308282EB422D401B701D6014630840095
:100680000008A20037087025840AB70A053037062B
:10069000031D402B3722B425F82D32261030D5000B
:1006A0003327D50B502B0800D6197B2B5618772BE8
:1006B000D6187A2BD408031D642B10304A1A622BEB
:1006C0004A1CC206CC060800D4180800541C0800B6
:1006D0004C164A186F2B4A1A712B4A16EC2A4A10EC
:1006E000732B4A124A1442124A1C4216EC2A641412
:1006F000E6010800FD290830CC065229D619A22BA4
:100700005618A12BD618A12BD408031D8E2B103000
:10071000CA1A8C2BCA1CC306CD060800D4180800C0
:10072000541C08004D16CA18992BCA1A9B2BCA16BE
:10073000EC2ACA109D2BCA12CA144312CA1C4316B3
:10074000EC2ACB290830CD065229D619C92B5618C8
:10075000C82BD618C82BD408031DB52B10304A1B44
:10076000B32B4A1DC406CE060800D4180800541C3A
:1007700008004E164A19C02B4A1BC22B4A17EC2AF6
:100780004A11C42B4A134A1544124A1D4416EC2A36
:10079000C5290830CE065229D619F22B5618EF2B50
:1007A000D618EF2BD408031DDC2B1030CA1BDA2B14
:1007B000CA1DC506CF060800D4180800541C08003E
:1007C0004F16CA19E72BCA1BE92BCA17EC2ACA1104
:1007D000EB2BCA13CA154512CA1D4516EC2A581828
:1007E0008B2AB12A0830CF065229D619102C561858
:1007F0000F2CD6180F2CD418042C20304A1A803015
:10080000C2060130EE06080039275208B100EE2674
:100810003927002739270130B100EE26392FC029AA
:100820000430CC065229D619282C5618272CD61855
:10083000272CD418222C2030CA1A8030C30602304C
:10084000EE06080039275008D3000027392F7029F9
:100850000430CD065229D6193F2C56183E2CD618F6
:100860003E2CD4183A2C20304A1B8030C406043069
:10087000EE06080039272A272A27392F7329043042
:10088000CE065229D619562C5618552CD618552C4A
:10089000D418512C2030CA1B8030C5060830EE0613
:1008A0000800392712271227392F76290430CF065E
:1008B0005229D619832C5618822CD618822C5418FB
:1008C000732CD418762C1F304A1C0F304A1A7F30F4
:1008D000500603190800D00A4A1C712C1030C206B9
:1008E000421EC20A0800C60AEC220800D00AFF30E5
:1008F00050060319AD0AD30A53197F2C222BD301BA
:10090000D20A222BB4290130CC065229D619A72CA1
:100910005618A62CD618A62C5418A02CD418A32CE4
:100920001F30CA1C0F30CA1A7F3051060319080045
:10093000D10ACA1C9E2C1030C306431EC30A0800ED
:10094000C70AEC220800D10A222B080072290130C4
:10095000CD065229D619C72C5618C62CD618C62C27
:100960005418C42CD41808001F304A1D0F304A1BDD
:100970007F30520603190800D20A4A1DC22C1030DB
:10098000C406441EC40A0800C80AEC2A75290130AE
:10099000CE065229D619E72C5618E62CD618E62C86
:1009A0005418E42CD41808001F30CA1D0F30CA1B7D
:1009B0007F30530603190800D30ACA1DE22C1030F9
:1009C000C506451EC50A0800C90AEC2A7829013067
:1009D000CF065229D6191A2D5618192DD618192DA9
:1009E0005418FF2CD418022D500803190800D00306
:1009F0004A1CFD2C1030C206421AC2030800C6036E
:100A0000EC220800D30353190F25D003FE30500603
:100A10000319AD03FF302D0603191325222B0330D4
:100A2000D300D20308000230AD07D3008030D200DB
:100A3000080079290230CC065229D619372D5618CC
:100A4000362DD618362D5418322DD418342D510881
:100A500003190800D103CA1C302D1030C306431AF5
:100A6000C3030800C703EC2AD103222B71290230EB
:100A7000CD065229D619522D5618512DD618512D62
:100A800054184F2DD4180800520803190800D20337
:100A90004A1D4D2D1030C406441AC4030800C80373
:100AA000EC2A74290230CE065229D6196D2D56181B
:100AB0006C2DD6186C2D54186A2DD41808005308C4
:100AC00003190800D3031030CA1D682DC506451A46
:100AD000C5030800C903EC2A77290230CF06522942
:100AE000A6008925220603190800260883169B0004
:100AF0001C158B138312220883169A0055309D0013
:100B0000AA309D009C149C18832D1C118B178312F6
:100B1000080083169B001C141A088312A900080001
:100B20003626B701B501370805201A26B70AB71DC2
:100B3000932D36269E25D327B425F82D80303226D6
:100B4000B70137086C20B70A003E0319A92D1A26F1
:100B5000A12DC0303226B70137087E20B70A003EEB
:100B6000031908001A26AC2D803032264C301A2684
:100B70006F301A2663301A263A301A26460828267D
:100B80002D304C1A2A301A26470828262D304D1AA7
:100B90002A301A26480828262D304E1A2A301A26BE
:100BA000490828262D304F1A2A301A2E8030322636
:100BB0004C301A26460828262D304C1A2A301A2680
:100BC0004C301A26470828262D304D1A2A301A266E
:100BD0004C301A26480828262D304E1A2A301A265C
:100BE0004C301A26490828262D304F1A2A301A2E42
:100BF000C03032267E306E187F301A2650082C26E0
:100C00007E30EE187F301A2651082C267E306E1961
:100C10007F301A2652082C267E30EE197F301A2695
:100C200053082C2EB400340E0F3930381A263408ED
:100C30000F393038B2002830A300A30B1D2E202618
:100C4000B20E32080F39350486008514851008006D
:100C5000BC009E272A08122EBC009E2728081826B2
:100C60002A08122E35121A26351608002830A3003D
:100C70009630B700C727A30B382E08002F08202076
:100C8000C111D408031D080056180800B425F82D1A
:100C9000051D502E8519542ED408031D44293B2AC6
:100CA000D408031D4429ED28C11C5E2EAE0B08009C
:100CB000C1103230AE000C30E20008009726EF3051
:100CC000A40006080B10A40C031C802E2408860028
:100CD00000000B1C612E4118772E4114060EA70050
:100CE0008226AF00C1140430AE00C115A12EAE0B98
:100CF000A12E0C306202031DE2036208AE00752EC5
:100D00004110762EA001A41D8C2EA00A241D8C2E2D
:100D1000A00AA41C8C2EA00A271C0E28A71C952E06
:100D2000271D932E2015A0150E2820150E28060825
:100D3000B600FF30860083168113F03086008312E0
:100D40000800360886008316811786018312080082
:100D50005B27B426BF2E5B27B626C32E5B27B8269B
:100D6000C72E5B27BA26CB2E4608BB2E4708BB2EC4
:100D70004808BB2E4908BD00B90068278F2F4208DC
:100D80004A1AD42ECE2E4308CA1AD42ECE2E440888
:100D90004A1BD42ECE2E4508CA1BD42EBE00B90045
:100DA0006827BF01C001752FBF003F30BE00B900EA
:100DB00068278F273F08B9006827D22E5B27B42603
:100DC0004C08CE2E5B27B6264D08CE2E5B27B826C4
:100DD0004E08CE2E5B27BA264F08CE2E0630B30023
:100DE00059277D30B900BD0068278F273108BE0024
:100DF000B9006827BF01C0017527B30BF02E0800AA
:100E00000630B300592753087F397838B900BD0040
:100E100068278F275108BE00B90068277527B30BD4
:100E2000022F08005B27B901BD0168278F27EC302E
:100E3000BE002D183E14AD18BE14B90068278F27C8
:100E40005008BF00B90068278F275108C000B900BB
:100E50006827752F5927BE017C30BD002D183D1421
:100E6000AD18BD141D2F20301A2E0512372F051670
:100E700008001430B2005B27B901BD01BE0168272C
:100E80008F27B9016827BF01C0017527B20B3B2F1F
:100E900008005B27FF30B900BD0068274F2F502F97
:100EA000512F00008F27B901BE016827BF01C00183
:100EB000752F19305C2F0F30A3005E2F5F2F0000BD
:100EC0008427A30B5D2F642F652F662F00008F2FC3
:100ED0000830BB000310B91F732F84276F2FB90D83
:100EE000BB0B6B2F08008F276F2F8F273D083E0607
:100EF0003F064006B90068278427BF01C001D40817
:100F00000319BD208F2F0800852F0330B700C72796
:100F10009B278A2F00000430B700C7279B2F902FF4
:100F200000000730B700C7279B270830972F982F5E
:100F3000B700C7279B2F013085060800031010302B
:100F4000BA00A501A801AA01BC0DAC0DAA0DA80DFF
:100F5000A50DBA0BAC2F00342A30B3272830B327A5
:100F60002530B327A42F840003300007A100A11966
:100F7000800030300007A100A11B8000003437083A
:100F8000D500C8303708C727D50BC12F0034000063
:100F9000C92FCA2F0130B8000000CE2FB80BCC2FBC
:100FA000B70BCA2F00340A30A5003230B700BF2774
:060FB000A50BD52F08007F
:02400E00303F41
:1042000003000400050006000F000000000000008D
:10421000000000000000000000000000000000009E
:10422000000000000000000000000000000000008E
:10423000000000000000000000000000000000007E
:10424000000000000000000000000000000000006E
:10425000000000000000000000000000000000005E
:10426000000000000000000000000000000000004E
:10427000000000000000000000000000000000003E
:10428000000000000000000000000000000000002E
:10429000000000000000000000000000000000001E
:1042A000000000000000000000000000000000000E
:1042B00000000000000000000000000000000000FE
:1042C00000000000000000000000000000000000EE
:1042D00000000000000000000000000000000000DE
:1042E00000000000000000000000000000000000CE
:1042F00000000000000000000000000000000000BE
:00000001FF
